:020000040000FA
:020000000528D1
:040002000034003492
:0800080009008C0123008C01AA
:1000100021006A30990021000F308C0020008B01F4
:100020008C01AE01A201A301A401A501A601A701B3
:10003000A001A1010C192D280C192F280030200235
:1000400003191A280830200203183328A10A0C309B
:10005000210203193628A0011A2800000000000020
:100060000000A00A1A28A001A1011A28A001A101DC
:100070000C1946280C19482800302002031938288A
:100080000830200203184C28A00138280000000086
:1000900000000000A00A382896019701A001A101E4
:1000A000A1150C1964280C196628003020020319C8
:1000B00051280830200203186A28A20D2214A10B2F
:1000C00062286E28A00151280000000000000000F6
:1000D000A00A5128A20D2210A10B6228A001A101A3
:1000E0000C197E280C198028003020020319702872
:1000F0000830200203188428A00112280000000004
:1001000000000000A00A7028A001A101A1150C198F
:100110009A280C199C2800302002031987280830DF
:1001200020020318A028A30D2314A10B9828A428AB
:10013000A00187280000000000000000A00A872816
:10014000A30D2310A10B9828A001A1010C19B4281C
:100150000C19B628003020020319A6280830200206
:100160000318BA28A00112280000000000000000B7
:10017000A00AA628A001A101A1150C19D0280C19CC
:10018000D228003020020319BD28083020020318AD
:10019000D628A40D2414A10BCE28DA28A001BD284E
:1001A0000000000000000000A00ABD28A40D2410DB
:1001B000A10BCE28A001A1010C19EA280C19EC28EA
:1001C000003020020319DC28083020020318F02830
:1001D000A0017C290000000000000000A00ADC282B
:1001E000A001A101A1150C1906290C19082900303C
:1001F00020020319F3280830200203180C29A50D4A
:100200002514A10B04291029A001F32800000000E7
:1002100000000000A00AF328A50D2510A10B042959
:10022000A001A1010C1920290C192229003020025B
:10023000031912290830200203182629A0017C295D
:100240000000000000000000A00A1229A001A10186
:10025000A1150C193C290C193E2900302002031964
:1002600029290830200203184229A60D2614A10BC3
:100270003A294629A00129290000000000000000B9
:10028000A00A2929A60D2610A10B3A29A001A10137
:100290000C1956290C195829003020020319482935
:1002A0000830200203185C29A0017C29000000000E
:1002B00000000000A00A4829A001A101A1150C1905
:1002C00072290C1974290030200203195F290830A3
:1002D000200203187829A70D2714A10B70297C2967
:1002E000A0015F290000000000000000A00A5F29B3
:1002F000A70D2710A10B7029220823062406250626
:1003000026062706031D122800307022A90001309E
:100310007022AA0003307022AB002308FE39A80027
:1003200022082906031DAF2928082A06031DAF2924
:10033000C2222318A5298C120000D22200000C161C
:100340002B1C1228B2220C1212280C120000D222EE
:1003500000008C162B1C1228B2228C1212282209A3
:10036000031DB429AE01122822080319592AA21B21
:10037000BF297039703A0319CE29AE011228AE0197
:100380001228EC302302031D12280730240603191B
:100390007B2A2508B0002408602210282E1CBD29C5
:1003A000A5080319162A2208783A0319E029220819
:1003B000743A0319FE2922087C3A0319062A1228E6
:1003C000241A122823087022AF00F121AF05A41DC2
:1003D000ED292F08031D9A2212282F0803199A22AB
:1003E000122801308A0024080739820701340234B8
:1003F000043408341034203440348034230870220C
:100400002402031D1228AE019A2212280730230667
:10041000031D0F2A08302406031D972A7F2A24086B
:10042000B00023086022AE019A221228221D272A3A
:10043000A2181228221C442A1D2A2308AC00AC034F
:100440000310AC0D0310AC0DAE149A221228AE1C92
:100450001228220803392C07AD0007302D06031996
:10046000762AA21D3B2A2308B0002D086022AD0188
:10047000AE019A2212282D0870222302031D122891
:10048000AD01AE019A221228AE1C1228A21D502ADC
:100490002308B0001C306022AC01AE019A22122861
:1004A0001C3070222302031D1228AC01AE019A22D7
:1004B000122822082306031D12282E148C0112284C
:1004C00023009100200030082300930015155530BB
:1004D0009600AA309600951495186C2A2000080002
:1004E000230091001514130820000800083023068B
:1004F000031D972A7F2A08302506031D1228810034
:10050000F8001E0000000000000020001D008130E7
:10051000B00000306022F830B000013060220A30B4
:10052000B000023060220130B00003306022AC0124
:100530002E1010288C120C16AA22AA22AA22AA2255
:10054000AA22AA220C12080000000230B100B10B4E
:10055000A72A08004730B200A422AE2AB20BAC2A68
:100560000000080002307022B6000A30B400C83023
:10057000B50000000000B50BB92AB40BB72AB60BC2
:10058000B52A080004307022B6000A30B400C83022
:10059000B50000000000B50BC92AB40BC72AB60B82
:1005A000C52A08001430B50000000000B50BD42A9D
:0205B000080041
:020000040001F9
:02000E00A40943
:02001000FF1CD3
:10E000008100F8000A0001000100000009009C00E6
:00000001FF
